:04000000D9EF03F041
:1000080000C015F09EA433D028D0BECF20F0BFCFBB
:1000180021F020C023F021C024F0BD6A040EBD6E7B
:1000280025C01CF023D0BECF20F0BFCF21F020C0C8
:1000380025F021C026F0BD6A050EBD6E27C01CF054
:1000480015D0BECF20F0BFCF21F020C027F021C0AF
:1000580028F09D9423C01CF009D01C50000AD5E05C
:100068001C50010AE0E01C50020AEBE09E9415C007
:0400780000F0110083
:10007C000F0E0C6E470E0D6E0D2EFED70C2EFCD7F0
:06008C000000000012005C
:0A009200210E0D6E0D2EFED7120098
:06009C000000000012004C
:1000A2000B840BAE5CEF00F0010E036E026A016A74
:0A00B200006A0A360232FF0E120047
:0800BC000AAE029E000E1200C4
:1000C4004FBE02D08C9E01D08C8E4FBC02D08C9C33
:1000D40001D08C8C4FBA02D08C9A01D08C8A4FB844
:1000E40002D08C9801D08C8822B002D08D8401D0AB
:1000F4008D948D82D1DF8D924FB602D08C9E01D02B
:100104008C8E4FB402D08C9C01D08C8C4FB202D018
:100114008C9A01D08C8A4FB002D08C9801D08C88F4
:1001240022B002D08D8401D08D948D82B5DF8D9262
:0C01340022A002D0A1DF01D0AADF12003F
:0E014000026A016A006A086A036A000E120071
:10014E00086A096A100E0C6E01340836093604501E
:10015E00085E0550D8A0053C095ED8B007D0045003
:10016E0008260550D8B0053C0926D8900036013631
:06017E000C2EEAD712006E
:100184000C6A0E6A0250D8A4DBEF00F001C002F042
:1001940000C001F0006A0E860250D8A4DBEF00F024
:1001A40001C002F0016A0E960E880250D8B4EDEF39
:1001B40000F00E50035ED8A4D8A0F2EF00F0D8905F
:1001C40002BEF7EF00F0003601360236032EE2EFEE
:1001D40000F0F2EF00F0010E0C6EB0DFFAEF00F069
:1001E400020E0C6E5CDFFAEF00F0040E0C6E64DF9E
:0201F4001200F7
:1001F6000B820BAE05EF01F0036802680168006828
:080206000A360232FF0E12005D
:0C020E0022904EC04FF057DF22801200FB
:08021A000B6A0B86FF0E1200B7
:100222000B800BAE1DEF01F0026A0AAEFF0E026EEA
:0C023200016E006E0A360232FF0E120050
:10023E000900F5CFE6FF0006FBE10106F9E1120029
:08024E00F28EF28CD08E12003A
:10025600BD6A050EBD6E9E949F849D849484130E84
:0A026600CD6ECF6ACE6ACD80120083
:0C0270000F0EC112936A94848284120065
:10027C00969296949598959A959C959E8D928D9420
:10028C008C9E8C9C8C9A8C98F3DEF2DEF1DE8C8A40
:10029C008C888D82FDDE8D92EBDE8D82F9DE8D9267
:1002AC00E7DE8D82F5DE8D92E3DE8C988D82F0DEBA
:1002BC008D92DEDE8D82ECDE8D928C9A8C8E8D8210
:1002CC00E7DE8D92D5DE8C9E8C888D82E1DE8D9260
:1002DC008C988D82DDDE8D92CBDE8D82D9DE8D9277
:1002EC008C888D82D5DE8D92C3DE8C988D82D0DE8B
:1002FC008D928C8E8C8C8C8A8C888D82C9DE8D92A2
:06030C00B7DE22801200A2
:100312000FD0800E476E19D0C00E476E16D0940EC5
:10032200476E13D0D40E476E10D0800E476E0DD09C
:100332004750010AEEE04750020AEEE04750030A36
:10034200EEE04750040AEEE0F0D74804006E475052
:10035200002600C047F000C04FF0B3DE22904B6A87
:100362004B504924E96E000E4A20EA6EEE520BE031
:100372004B504924E96E000E4A20EA6EEECF4EF051
:0A03820045DF4B2AEDD72280120060
:10038C000B6A0C6A0A6A0350D8B410EF02F0028EA2
:10039C008E0E035E03BED8EF01F0D8B4D8EF01F097
:1003AC0014EF02F0036C080E035CD8A0EFEF01F021
:1003BC00036E013602C001F0026A080E035CD8A07D
:1003CC00EFEF01F00136016A0350D8A4D890F9EF91
:1003DC0001F00350D8B4F9EF01F0D8900232013299
:1003EC00032EF3EF01F00BBC01A006EF02F0D8A036
:1003FC0006EF02F0012AD8B4022A02BE23EF02F063
:10040C000AAE28EF02F0021E011E012AD8B4022AFD
:10041C0028EF02F0026A016A28EF02F00B800BAEA3
:10042C002CEF02F0026A0AAE2CEF02F0FF0E026E05
:10043C00016E0A3602322CEF02F0010E0C6EEBDE6E
:10044C002EEF02F0000E0C6E2EEF02F0FF0E0C6E73
:0A045C000150006E0250016E120004
:100466004B6A050E4B5C0AE24B504924E16E000EC6
:100476004A20E26E200EE66E4B2AF3D74B504924F3
:10048600E16E000E4A20E26EE66A4B064B504924A6
:100496004C6E000E4A204D6E0A0E046E000E056E5E
:1004A60047C000F048C001F04FDE08C000F009C0A8
:1004B60001F0300E00264CC0E1FF4DC0E2FF00C047
:1004C600E6FF0A0E046E000E056E47C000F048C037
:1004D60001F03ADE00C047F001C048F0000E0118F6
:1004E60002E1000E001801E102D04B06CFD7120040
:1004F600086A096A000E0762036400EF03F00250FF
:1005060006180A6E075003267E0ED8A091EF02F059
:10051600035ED8B004EF03F095EF02F0035ED8A0B7
:1005260008EF03F0028E068E02C00EF001C00BF03B
:1005360000C00DF000500402F4CF0CF0015005028B
:10054600F4CF00F0F3CF08F00402F3500C26F45079
:100556000822000E00220D500502F3500C26F4501E
:100566000822000E002202500402F3500826F4501E
:10057600002202500502016A000E0122F3500026F5
:10058600F45001220D500602F3500826F4500022C2
:10059600026A000E012202220B500602F3500026C8
:1005A600F4500122000E02220E500602F3500126DC
:1005B600F450022202BEE8EF02F008360036013699
:1005C60002360306D8B408EF03F0FBEF02F0D8803A
:1005D600800E08640030000E002201220222D8A0FC
:1005E600FBEF02F0023201320032034A04EF03F05D
:1005F6000AAE029E000E0AEF03F0010E9EDD0AEF20
:1006060003F0020EF5DD0AEF03F0040E47DD1200DB
:100616000050086E0150006E016A026A036A0B6A96
:100626000C6A960E036E0A6A00C001F008C000F05C
:08063600086A026AA4DD12004B
:10063E000450000A12E10550000A0FE10650000AAC
:10064E000CE10750000A09E1FF0E006EFF0E016E6D
:10065E007F0E026EFF0E036EA4D0086A096A075061
:10066E00D8B4CAEF03F00350D8B4CEEF03F0025063
:10067E0006180A6E028E068E0E6A02C008F001C0BF
:10068E000CF000C00DF004500D5E0550D8A0053CD6
:10069E000C5E0650D8A0063C085E086A0C6A0D6A0D
:1006AE00D8A061EF03F0D890023201320032083246
:1006BE00010E0E6E0750035ED8A06EEF03F07E0E95
:1006CE000E240326D8B0D2EF03F074EF03F07E0EA3
:1006DE000E240326D8A0D6EF03F0180E0B6E0D369F
:1006EE000C3608360036013602360E360450005EE1
:1006FE000550D8A0053C015E0650D8A0063C025E0F
:10070E0006340E120EA08FEF03F00D809AEF03F059
:10071E00045000260550D8B0053C01260650D8B02E
:10072E00062802260D900B2E76EF03F0C0EF03F095
:10073E00D8900036013602360E360450005E055053
:10074E00D8A0053C015E0650D8A0063C025E0634D9
:10075E000E10010B0D26D8B00C2AD8B4082AD8A436
:10076E00C0EF03F008320C320D32032AD8B4D2EFA8
:10077E0003F00AAE089E0850026E0C50016E0D502A
:10078E00006ED8EF03F0010E41DDD8EF03F0020E3C
:10079E00D0DCD8EF03F0040E27DDD8EF03F0080EFF
:0407AE0079DC1200E0
:1007B200440E166E3A0E176E186A500E196E3A0EE5
:1007C2001A6E1B6A1C6A570E1D6E3A0E1E6E1F6A47
:1007D2003F6A406A4CDD3ADD3DDD4FDD010E4F6E72
:1007E20070DC0C0E4F6E6DDC010E476E010E486E12
:1007F200160E496E000E4A6E8BDD010E476E090E13
:10080200486E1D0E496E000E4A6E82DD020E476E64
:10081200090E486E190E496E000E4A6E79DD9DB4BE
:1008220082D02350255C006E24502658016E00C0F1
:1008320029F001C02AF02350275C456E2450285825
:10084200466E45C03FF046C040F0E4DE00C041F0D5
:1008520001C042F002C043F003C044F045C000F0C2
:1008620046C001F0D7DE00C004F001C005F002C0AE
:1008720006F003C007F041C000F042C001F043C0DF
:1008820002F044C003F0DADE000E046E000E056EC4
:10089200480E066E850E076E2DDE77DD00C047F02E
:1008A20001C048F02B0E496E000E4A6EDBDD010ED0
:1008B200476E030E486E2B0E496E000E4A6E28DDFF
:1008C20029C047F02AC048F02B0E496E000E4A6E2E
:1008D200C9DD010E476E0B0E486E2B0E496E000EDF
:1008E2004A6E16DD3FC047F040C048F02B0E496EFD
:1008F200000E4A6EB7DD020E476E0B0E486E2B0ECF
:10090200496E000E4A6E04DD040E0B6E0C0E0C6E68
:10091200330E0D6E0D2EFED70C2EFCD70B2EFAD7F2
:0A092200000000009D847BD7FFD782
:020000040030CA
:0D000100021F1EFF8181FF0FC00FE00F40A6
:00000001FF
